:020000040800F2
:100000000010002089120008C9080008CB08000869
:1000100000000000000000000000000000000000E0
:10002000000000000000000000000000CD080008F3
:100030000000000000000000CF0800088112000846
:10004000D912000800000000D9120008D9120008D7
:10005000D9120008D9120008D1080008DB080008EE
:1000600000000000E5080008F50800080509000880
:1000700015090008D9120008D91200080000000074
:10008000D912000800000000000000002509000847
:1000900000000000D9120008D9120008D912000887
:1000A00000000000D9120008000000003509000817
:1000B0000000000000000000000000000000000040
:1000C00010B5064C2378002B07D1054B002B02D02E
:1000D000044800E000BF0123237010BD1000002081
:1000E0000000000050380008044B10B5002B03D06E
:1000F0000349044800E000BF10BDC04600000000F6
:1001000014000020503800080023C25C0133002A8C
:10011000FBD1581E7047000002B4714649084900DF
:10012000095649008E4402BC7047C04602B471466D
:1001300049084900095C49008E4402BC7047C0462A
:10014000002243088B4274D303098B425FD3030A16
:100150008B4244D3030B8B4228D3030C8B420DD329
:10016000FF22090212BA030C8B4202D312120902B7
:1001700065D0030B8B4219D300E0090AC30B8B42F5
:1001800001D3CB03C01A5241830B8B4201D38B03A3
:10019000C01A5241430B8B4201D34B03C01A524148
:1001A000030B8B4201D30B03C01A5241C30A8B428B
:1001B00001D3CB02C01A5241830A8B4201D38B0276
:1001C000C01A5241430A8B4201D34B02C01A52411A
:1001D000030A8B4201D30B02C01A5241CDD2C3098C
:1001E0008B4201D3CB01C01A524183098B4201D308
:1001F0008B01C01A524143098B4201D34B01C01AF3
:10020000524103098B4201D30B01C01A5241C3086A
:100210008B4201D3CB00C01A524183088B4201D3D9
:100220008B00C01A524143088B4201D34B00C01AC5
:100230005241411A00D20146524110467047FFE731
:1002400001B5002000F0F0F802BDC0460029F7D04B
:1002500076E7704703460B437FD4002243088B4266
:1002600074D303098B425FD3030A8B4244D3030B3D
:100270008B4228D3030C8B420DD3FF22090212BA02
:10028000030C8B4202D31212090265D0030B8B427E
:1002900019D300E0090AC30B8B4201D3CB03C01A68
:1002A0005241830B8B4201D38B03C01A5241430B43
:1002B0008B4201D34B03C01A5241030B8B4201D333
:1002C0000B03C01A5241C30A8B4201D3CB02C01A9E
:1002D0005241830A8B4201D38B02C01A5241430A16
:1002E0008B4201D34B02C01A5241030A8B4201D305
:1002F0000B02C01A5241CDD2C3098B4201D3CB01AC
:10030000C01A524183098B4201D38B01C01A52415A
:1003100043098B4201D34B01C01A524103098B425E
:1003200001D30B01C01A5241C3088B4201D3CB0049
:10033000C01A524183088B4201D38B00C01A52412C
:1003400043088B4201D34B00C01A5241411A00D2DC
:1003500001465241104670475DE0CA0F00D0494245
:10036000031000D34042534000229C4603098B42B5
:100370002DD3030A8B4212D3FC22890112BA030A3D
:100380008B420CD3890192118B4208D389019211BF
:100390008B4204D389013AD0921100E08909C30944
:1003A0008B4201D3CB01C01A524183098B4201D346
:1003B0008B01C01A524143098B4201D34B01C01A31
:1003C000524103098B4201D30B01C01A5241C308A9
:1003D0008B4201D3CB00C01A524183088B4201D318
:1003E0008B00C01A5241D9D243088B4201D34B0033
:1003F000C01A5241411A00D20146634652415B1075
:10040000104601D34042002B00D549427047634655
:100410005B1000D3404201B5002000F005F802BD9A
:100420000029F8D016E770477047C046D0400B004F
:10043000D1409C46203AD3401843524263469340F1
:100440001843704730B585B00C22002101A803F095
:10045000F6F90422164C174B626180222360802338
:100460005202A261C2221B06012563600023FF32F3
:10047000E2612000621DA360E36025612362D377FF
:10048000A56201F021F8002801D000F003FA8023D2
:100490005B0102930723200001A90195039301F05A
:1004A00001FA002801D000F0F5F905B030BDC046D2
:1004B0002C0000200024014030B5050089B0142232
:1004C000002103A803F0BBF9214B2A689A423CD1D2
:1004D0008020204B800099690143996180219A69AD
:1004E000890202400192019A5A6990200A435A6196
:1004F0005B69C0050B400293029B022303A903938F
:100500000133049301F0ACFC8022134C134BE260E6
:10051000921822618022D20023606261002320228F
:1005200020006360A360A261E36101F083FA002808
:1005300001D000F0AFF900220C2011002C6365629D
:1005400001F028FA0C2001F04FFA09B030BDC04686
:1005500000240140001002406C000020080002400E
:1005600013B50124104B21005A69092022435A6116
:100570005B69002223400193019B01F00BFA0920E3
:1005800001F032FA210000220A2001F003FA0A20C9
:1005900001F02AFA002221000B2001F0FBF90B20C8
:1005A00001F022FA13BDC0460010024030B589B0F8
:1005B0001422002103A803F042F980202F4BC0032E
:1005C00059699025014359615A69ED05024080201F
:1005D0000092009A596980020143596180215A6949
:1005E000C90202400192019A5A6928000A435A61DD
:1005F0005B6901220B4002931021029B01F0ECFC8D
:1006000000222800202101F0E7FC08230393C423E3
:10061000002428009B0303A90493059401F020FC07
:1006200030232800039303A92F3B049306930594DA
:1006300001F016FC4023280003A9039304940594B9
:1006400001F00EFC80230393882328005B0303A999
:100650000493059401F004FC22000221062001F01D
:1006600099F9062001F0C0F922002100072001F0CD
:1006700091F9072001F0B8F909B030BD001002402F
:100680000848094B10B5036006234360074BC3605D
:100690009C239B00836001F0B9FC002801D000F08E
:1006A000F9F810BDB000002000300040FF0F00003E
:1006B00030B595B0282200210AA803F0C0F8102216
:1006C0000021684603F0BBF81022002104A803F0C3
:1006D000B6F80923089380235B0211938023012439
:1006E00002255B0308A809940F941095129301F05A
:1006F000C7FC002801D072B6FEE7072302900390E2
:10070000210068460093019501F0ECFE002801D01D
:1007100072B6FEE7069004A8049401F077FF002863
:1007200001D072B6FEE715B030BD0000F8B500F09C
:10073000F9FDFFF7BDFFFFF739FFFFF711FFFFF7E7
:1007400081FE00F0A3F9FFF79BFF00F065F9414B34
:1007500041481988414A4B1E9BB283426FD8118091
:100760003F4B19883F4B4A1E92B282426AD8198089
:100770003D4C1B88226853633C4B3D4A19884B1CF7
:100780009BB2012B62D911803A4E300001F070FC0F
:10079000200002F071F80021200002F0E3FA364C4C
:1007A000200002F06FFB20222000344902F0E4FF19
:1007B000334F344CFA223900200000F02DFF9020F6
:1007C00000222021C00501F007FC3221002000F0AA
:1007D00015FDFA210120490000F010FD02202A49F0
:1007E00000F00CFD002000F01FFD002809D02000C3
:1007F00000F05CFF00F0EAF9FA223900200000F076
:100800000BFF012000F010FD002807D0300001F0A0
:100810002FFC90201021C00501F0E4FB022000F025
:1008200003FD002802D00222184B1A70184D2B78B5
:10083000002BD7D000F0CCFB00232B70D2E7012394
:1008400013808DE7FA2292001A8091E70A23138021
:100850009AE7C046003C0008FDFF0000140200209B
:10086000023C00085A040020C0000020043C00089C
:100870004C040020B0000020900100200A04002059
:10088000160200202C000020881300000400002025
:100890007C04002072B6FEE701200A4B82B0996901
:1008A0000143996180219A69490502400092009AAA
:1008B000DA690A43DA61DB690B400193019B02B0FC
:1008C0007047C04600100240FEE7FEE770477047E1
:1008D00010B5082001F08EFB10BD10B5802001F08E
:1008E00089FB10BD10B5024801F055F910BDC04696
:1008F0006C00002010B5024801F04DF910BDC04653
:100900000801002010B5024801F045F910BDC046AD
:100910004C01002010B5024800F054FF10BDC04645
:100920002C00002010B5024801F0D4FF10BDC046D5
:10093000C000002070B5114C200002F069FB2000BF
:1009400002F0A0FA102223680D4DD96911420FD090
:100950001A620C4B1A78002A0AD10B4A0B4812680B
:1009600051682022521AD2B229001A7002F05EFF9A
:1009700029002022200002F0FFFE70BD900100201F
:100980000A0400207C040020080100205C040020F0
:100990007047000007B50B4B02689A4211D18020C6
:1009A000094A4000D1690143D161D3690121034063
:1009B0000193ED380022019B00F0ECFF132001F0C1
:1009C00013F807BD002000400010024010B50400DD
:1009D00086B01422002101A802F031FF0B4B2268DF
:1009E0009A4210D180200A4AC002516901435161E4
:1009F000536901A903400093009B0223054801931A
:100A0000029301F02DFA06B010BDC0460020004050
:100A1000001002400004004810B588B01C220021DC
:100A200001A802F00CFF164C164B174A2360012355
:100A3000636000232000A360E2602361A36102F0F1
:100A40002DF8002801D0FFF725FF200002F04EF816
:100A5000002801D0FFF71EFF602300220193200031
:100A6000CC3301A902930392059202F0A3F8002867
:100A700001D0FFF70FFF2000FFF7A8FF08B010BD5F
:100A8000C000002000200040E70300000B480C4B92
:100A900010B5036096239B010C2243600023426142
:100AA0008360C36003618361C3610362436202F0D8
:100AB000DDFD002801D0FFF7EDFE10BD9001002004
:100AC0000038014030B5050089B01422002103A888
:100AD00002F0B5FE354B2A689A4265D18020344B2E
:100AE000C00199690143996180219A698902024094
:100AF0000192019A5A6990200A435A615B69C005C4
:100B00000B400293029BC023DB0003930223049358
:100B10000133069303A9023B079301F0A1F9254C89
:100B2000254B8022236000236360A36023616361FF
:100B3000A361802320005B01E260E36100F07AFFA3
:100B4000002801D0FFF7A6FE1C4B2C6765621C4CE9
:100B500080222360102363600023A360236163610C
:100B6000A361802320005B01E260E36100F062FF8B
:100B7000002801D0FFF78EFE8023124A9B001168E7
:100B80001B200B4313600022EC661100656200F02D
:100B900001FF1B2000F028FF10220B4B1B68196877
:100BA0000A431A6050221A6209B030BD0038014071
:100BB00000100240080100203000024044000240C2
:100BC0004C010020000001409001002070B5244C31
:100BD0000121228813004800205A984239D8051C68
:100BE000904200D9151CAAB20131FA29F3D1991A01
:100BF000002904DD1B4908881B189B1A0B801A4C1E
:100C000023785A1C2270032B22D9164D052100236C
:100C1000E85EFFF71FFB03B2144815495843FFF77E
:100C200019FB144B0A2100229B5E5843FFF712FB6D
:100C3000114B1B785BB25843104B00B21880104B1D
:100C40001B78012B07D10F4B188000232B802370BA
:100C500070BD0300C8E7002BF7D10B4BF4E7C0468B
:100C6000160200204A04002057040020E40C000073
:100C7000FF0F00004C040020080000204E0400205C
:100C800055040020520400205004002010B5040038
:100C9000902001222021C00501F09EF909490A484F
:100CA000A2B202F093F8094800F0BEFF0128FAD181
:100CB000043000F0CDFA902000222021C00501F080
:100CC0008BF910BD2A040020900100204C01002067
:100CD00070B54D4C86B0A01C00F028FA0600201D0F
:100CE00000F024FA06210500200000F027FA020A8D
:100CF000D2B2C0B2012E34D1022D30D1A1799142AD
:100D00002DD1E27982422AD10022404B40499A56A5
:100D1000012A0BD100200B5ED8171B1843409620E8
:100D20009BB24000834201D25B420B80394D237855
:100D300028002B706378AA716B700423AB700023BA
:100D4000CB5E19122B711312E9706B71072100F041
:100D5000F5F9030A28720920EB71FFF797FF06B037
:100D600070BDFF2E17D0022E31D0032EF7D1012DEA
:100D7000F5D1A1799142F2D1E2798242EFD1254DAC
:100D800023782B7063786B700223AB70224B0022A8
:100D90009B5E1A122CE0012DE1D1A1799142DED1A6
:100DA000E2798242DBD1002401AD122228001B49E6
:100DB00002F03CFD174E2800FFF7A6F9844201D34C
:100DC000C0B2CAE72B5D33550134E4B2F3E7012D1D
:100DD000C5D1A1799142C2D1E2798242BFD10D4DF4
:100DE00023782B706378AE706B700D4B1B881A0ADA
:100DF0002B7105212800EA7000F0A0F9030AA87100
:100E00006B710720A9E7C0465C04002004000020A5
:100E10004E0400202A0400204C04002080380008E2
:100E20005A04002070B500230124174E86B00293A7
:100E300003930496059400F01BFF694603A801ADD7
:100E400000F0C4FF002819D1104B31001B8803307B
:100E50002B701B0A6B700E4B1B88AB701B0AEB7060
:100E60000C4B00229B5E2B711B126B71019A029B33
:100E700000F046FF041E04D100F00EFF200006B073
:100E800070BD0324FAE7C046003C000814020020AD
:100E90005A0400204C040020F7B5444C65792079B1
:100EA0002D020543A01C00F041F90621009020000E
:100EB00000F044F93E4F062201902100380002F074
:100EC000B5FC6A46019B10791B0A009A6DBADBB229
:100ED000AEB2BB71F8710F2A28D1A2799A4214D10F
:100EE000E379834211D1013EF62E14D8314B1D8097
:100EF000012383F31088FFF795FF002805D180F3C5
:100F0000108823780820002B2ED1202200212000D9
:100F100002F095FCF7BDFF2306213B717B71200099
:100F200000F00CF9030ABB71F871EAE7009A022A93
:100F30001DD1A2799A42E8D1E3798342E5D1FA2220
:100F4000731E9BB292009342DFD21B4B1D801B4B42
:100F50001B685E63012383F31088FFF763FF00289B
:100F6000D3D180F310880830FFF790FECDE7009AC8
:100F7000032ACAD1A2799A42C7D1E3798342C4D164
:100F80000F4BF6180F4BB6B29E42BED828B20E4E8B
:100F90000A25012807D00D4B68430021595EFFF751
:100FA00059F93080D6E73580D4E7C0465C0400208C
:100FB0002A040020140200205A040020C00000204F
:100FC000E40C0000C81900004C0400204E0400206E
:100FD00010B50F4B0F491A7809880F4C91420FD169
:100FE0002278082A09D15B78032B04D0062B04D180
:100FF000FFF752FF01E0FFF76BFE0023237010BDE7
:10100000002AFAD12278082AF7D15B78EEE7C046A9
:101010005C040020140200207C04002010B50400B1
:1010200080281DD190204021C00500F0CFFF01286D
:1010300003D1324A137801331370314A13780133E4
:10104000DBB21370092B0AD92C4B01211878022826
:1010500000D802392B48017000211170197010BDA1
:101060000828FCD10220284900F0C8F8902021006F
:10107000C00500F0ABFF2549254B264A012827D1A2
:10108000087000215B5E244912880024095F5B1A06
:10109000934210DD214A13780133DBB21370022B27
:1010A000DDD900211E4801701E480170FA2BD6D9E7
:1010B00003231370D3E71B4A13780133DBB2137099
:1010C000022BCCD916490870002014490870EDE7AE
:1010D0000020087000215B5ED9175B184B40124955
:1010E0009BB28B4202D95A231380B8E7FA214900F8
:1010F0008B4201D93C23F7E71E23F5E75804002073
:10110000540400200800002088130000550400202B
:101110005204002006000020500400205904002042
:101120000400002056040020DC050000027840780E
:101130000002104340BA80B270470000FF22130043
:10114000F0B5084D084E094F013989B2A94202D1C4
:1011500018021043F0BD047801305C40335D534009
:101160003A5DF1E7FFFF000092380008923900086D
:101170001C4A70B51368002B07D01368013B13603D
:10118000002B02D10122184B1A7000220C250126D7
:1011900016482C0054430319596800290AD059688D
:1011A00001395960002905D15E70215C012901D106
:1011B000996859600132042AEBD10D4B1A6801324B
:1011C0001A6019680B4A914201D100221A600A4A3A
:1011D00013780133DBB2092B01D8137070BD0023E3
:1011E000FBE7C046BC040020B804002088040020AF
:1011F00080040020FFFFFF7F84040020030030B53F
:10120000032800D9FEE7012585F310880C20002271
:101210005843044C2318596099605A70055582F35D
:10122000108830BD8804002003000020032B09D85B
:101230000C305843054B00221B185978C8B20129BD
:1012400001D15A7070471000FCE7C04688040020A6
:1012500000280FD0012800D10130012383F310882A
:101260000022054B1860054B1A7082F310881A781B
:10127000012AFCD17047C046BC040020B8040020FD
:1012800010B5FFF775FF10BD0D4885460D480E4996
:101290000E4A002302E0D458C4500433C4188C42D0
:1012A000F9D30B4A0B4C002301E013600432A24235
:1012B000FBD3FFF76DFB02F095FAFFF737FAFEE775
:1012C000001000200000002010000020C03A00089C
:1012D00010000020E8040020FEE7000070B50500C3
:1012E000FA200D4B80001978FEF72AFF0B4B010006
:1012F0001868FEF725FF00F083FB04000120002C96
:1013000009D1032D07D802382200290000F042FB42
:101310002000034B1D6070BD09000020000000206C
:101320000C0000201023064A10B5116803200B435F
:101330001360FFF7D3FFFFF7AFFA002010BDC046E0
:1013400000200240014B18687047C046C0040020CE
:101350000321036870B59A6804000A40012A01D08D
:10136000002070BD1968114202D1DA681204F7D565
:1013700005229D681540012D1ED19968033A0A4344
:101380009A6003221A60FFF7DDFF060023689B685E
:101390002B42E5D0FFF7D6FF801B0228F6D9236841
:1013A0009B682B42F2D01023A26B01201343A3634E
:1013B000E36B1D43E563D4E710230120A26B1343C5
:1013C000A363E36B0343E363CBE70000002373B540
:1013D00003210193036804009A680A40012A07D197
:1013E0001968114201D0002076BDDA681204FAD4DF
:1013F00099681B4A114208D010230120A26B1343A5
:10140000A363E36B0343E363EEE7012299680A43B6
:101410009A60144B14491868FEF792FE0190019BE4
:10142000002B19D1FFF78EFF0125060023681B68EA
:101430002B42D8D1FFF786FF801B0228F6D92368FC
:101440001B682B42F2D11023A26B01201343A3632C
:10145000E36B1D43E563C7E7019B013B0193DEE7B7
:10146000170000800000002040420F0004220368A3
:1014700070B599680400114201D1002070BD9968CF
:10148000114206D09A68920703D4102299680A4341
:101490009A60FFF757FF0426050023689B683342D4
:1014A000EBD0FFF74FFF401B0228F6D923689B685B
:1014B0003342F2D010230120A26B1343A363E36BEA
:1014C0000343E363DAE70000F8B504000120002CD1
:1014D00000D180E0A36B002B06D122003432E363FD
:1014E00020001370FEF7E8FFA36BDB0600D587E052
:1014F00023680422996808001040114200D07FE060
:10150000A26B4249114002220A430321A2639A6856
:101510000A40012A05D1196811420ED1DA68120475
:101520000BD41821DA688A43A1680A43DA60196982
:1015300062688900890811431961DA6834490A40F0
:10154000DA60A26A267E571E7A1E9741617EE268A3
:10155000C903B6030E43A57E1643226969033F0300
:101560000E43022A00D10420621DD27FE17E520088
:1015700032433A430243012904D1002D2CD180216A
:1015800049020A43C220E169FF30814202D0206A49
:1015900001430A438020D96840051143D960E16ABC
:1015A000814202D0481E062807D8072558692940DD
:1015B000A8435861586901435961DB6815490B40DC
:1015C000934211D100200322E063A36B93431A00DE
:1015D00001231343A363F8BD2020A56B2843A06318
:1015E000E06B0143E163CDE71222A36B012093433B
:1015F0001A0010231343A363E36B0343E363EAE797
:101600001023A26B01201343A363E4E7FDFEFFFF59
:101610001902FEFFE7FF3F83F7B5036804009B68EC
:101620000E00022001925B0730D4270034373B784C
:10163000012B2BD001233B70637E012B27D1A36BA1
:10164000164A00251A4080235B001343A363E56319
:101650003D70206B124B21688362124BC362124BA8
:1016600003631C230B604A680C3B13434B6001234C
:10167000CA681343CB603200019B403100F00CFA82
:1016800004232800226891680B439360FEBD20006C
:10169000FFF79CFE0028D2D0F8E7C046FEF0FFFF1F
:1016A000291700089B170008A9170008F8B50600BD
:1016B0003436337805000224012B24D001273770FB
:1016C000FFF7D4FE041E1CD12A68286BD368BB43E5
:1016D000D360831CDB7F022B07D100F01BFA041EB2
:1016E00003D04023AA6B1343AB6310212A68280060
:1016F00053688B435360002C07D1FFF729FE041E6B
:1017000006D0002333702000F8BDFFF721FEF8E774
:10171000AB6B034A1A4001231343AB63F1E7C046A6
:10172000FEFEFFFF704700005022436A10B5996B20
:1017300011422AD1996BB132FF320A43C0219A6318
:101740001A680901D068084212D1997E00290FD188
:10175000116809070CD5916849070DD40C20516810
:10176000814351609A6B0B49114001220A439A63ED
:101770001800FFF7D7FF10BD2022996B0A439A6328
:101780000122D96B0A43DA63F2E71B6B1B6B9847A4
:10179000F1E7C046FEFEFFFF704710B5406AFFF755
:1017A000FBFF10BD704770474023406A10B5826B45
:1017B000134383630423C26B1343C363FFF7F3FF35
:1017C00010BD00000422036870B5196804001142BE
:1017D00002D05968114206D108221968114228D056
:1017E0005968114225D0A26BD20604D48022A16B85
:1017F00092000A43A263C022D9681201114212D199
:10180000A27E002A0FD11A6812070CD59A685207D7
:101810003CD40C215A688A435A60A36B204A1A4070
:1018200001231343A3632000FFF77CFF0C222368EE
:101830001A60802523681A682A420CD05B682B4204
:1018400009D08023A26B5B021343A3632000FFF740
:10185000A9FF23681D60102223681968114214D063
:101860005968114211D0A26A012A02D0DA68D2075F
:1018700008D50222E16B20000A43E26310221A60BD
:10188000FFF791FF102223681A6070BD2023A26B1E
:101890001343A3630123E26B1343E363C3E7C0462F
:1018A000FEFEFFFFF0B50023040085B0039334343F
:1018B00023780200C66A0220012B2FD00138207045
:1018C000136804279D68AC463D40019565463D423E
:1018D00051D10F682A4D3A00AC464D68B840103AD5
:1018E000654537D09D6A284398628020400586422E
:1018F0000FD0013E062E0CD907205D69896805408E
:10190000A94206D05D69014085435D615D69294357
:101910005961012A04D900200023237005B0F0BDCD
:10192000184A80211368102F12D0C9030B4313608B
:10193000102FF0D1144B15491868FEF701FC0A234B
:1019400043430393039B002BE5D0039B013BF8E744
:101950000904EBE7996A81439962012ADBD8534273
:101960005A4152420749920D9305094A08689B184B
:1019700003400B60CFE72023916B0B439363CBE7CE
:1019800001100000082701400000002040420F0025
:10199000FFFFBFFF30B5FF2503242A000440E40009
:1019A000A24089012940D243A140C3B200280ADBEA
:1019B000C0240B4B80088000C018A40003591A40B3
:1019C0001143015130BD0F200340083B05489B08DF
:1019D0009B001B18D86902401143D961F2E7C04649
:1019E00000E100E000ED00E0002805DB1F231840C7
:1019F0001E3B8340014A13607047C04600E100E08F
:101A00008022431E5204012093420DD2C021074A76
:101A100007485360036A09061B021B0A0B43036253
:101A200000200723906013607047C04610E000E07C
:101A300000ED00E070B504000120002C24D002234A
:101A4000A51CEB772068114B0268A1681A406368F7
:101A50000B43E1680B4321690B4361690B43A169A7
:101A60000B43E1690B4313430360094B1421C01876
:101A7000FEF766FB074B80002064E3630020012330
:101A8000A063E418EB77E07770BDC0460FC0FFFF9E
:101A9000F8FFFDBF00000240F7B5451C0193EB7F46
:101AA00004000220012B27D001232718EB77FB7FAE
:101AB00000269C466046DBB2012828D10130F87729
:101AC0002068A6630568266C9D43B3400560E56BFE
:101AD0006B60019B43606368102B0ED18260C16014
:101AE000E36A0268002B0BD00E231343036001232B
:101AF0000268134303600020FEBD8160C260EFE70F
:101B00000A2313430422036003689343EEE7022091
:101B1000EE77F1E730B5851CEB7F441C022B05D036
:101B20000423836300230120E37730BD0E21036883
:101B30001A688A431A600122196891431960016C7E
:101B4000C36B1000884058600020EA77E077ECE72C
:101B500070B5841CE37F022B04D004238363033B12
:101B6000180070BD0E210368056C1A688A431A605C
:101B700001221968914319601100A940C36B596093
:101B8000E27700248318DC77426B1300A242E7D08F
:101B900090472300E4E7F8B504273E00016CC26BD0
:101BA0008E40156803681C6835420DD03C420BD04E
:101BB0001968890602D41968B9431960C36A566066
:101BC000002B19D0984717E002273E008E4035427F
:101BD00013D03C4211D01968890606D40A2419682A
:101BE000A14319600121C319D97756600022431C13
:101BF000DA77836A9342E5D1F8BD082637008F4033
:101C00003D42F9D03442F7D00E251C68AC431C602D
:101C100001231C008C405460821C8363D377002214
:101C2000C318DA77036BE5E70230C07FC0B27047B4
:101C3000806B70470C4A1021D06830B503000B4010
:101C4000084205D002230948C4692343C3610B003D
:101C50000420D168014205D00121044C0343E56909
:101C60002943E161D36030BD00200240C804002058
:101C7000064B00201A69120606D5054A5A60054A25
:101C80005A6018690006C00F7047C0460020024025
:101C900023016745AB89EFCD8023034A00201169FA
:101CA0000B4313617047C0460020024070B504002A
:101CB000FFF748FB01260500104BDA68324211D1CC
:101CC0002022D968114200D0DA60D96810220800B9
:101CD0001040114202D1DB685B0708D5FFF7AAFF6D
:101CE000012004E0621CE8D0002C01D1032070BD6B
:101CF000FFF728FB401BA042DED9F7E70020024097
:101D0000F0B585B003931C4B019102921A7E04003A
:101D10000220012A2ED0012218481A76FFF7C6FFAA
:101D2000002824D12600012C02D0022C00D0042649
:101D30000024029803992201FEF778FB0022012774
:101D40000D4B0F4DDA612B69019A3B432B61630008
:101D50009B1880B218800948FFF7A8FF2B69BB4386
:101D60002B61002803D1E419E3B29E42E1D800229E
:101D7000014B1A7605B0F0BDC804002050C3000026
:101D8000002002400022064BDA61064B043219693A
:101D90000A431A61402219690A431A617047C04612
:101DA000C8040020002002400022064BDA61064BE6
:101DB000023219690A431A614022586119690A43BB
:101DC0001A617047C804002000200240F8B5214F76
:101DD00004003B7E0E000220012B0CD001233B7639
:101DE00023681D48012B12D1FFF760FF002803D0A4
:101DF000012000233B76F8BDFFF7C4FF1648FFF72C
:101E000055FF0421154A13698B431361F1E7FFF76E
:101E10004DFF0028ECD101235B423360656801303F
:101E2000A36862689B029B18AB42E2D92800FFF7C7
:101E3000BBFF0948FFF73AFF0221084A13698B43A9
:101E40001361002801D03560D3E78023DB00ED1853
:101E5000E6E7C046C804002050C30000002002404E
:101E60000023F0B587B00A681400DC4001D107B048
:101E7000F0BD012514009D402C4001942A4200D160
:101E800095E04A685E00944603226446224003249B
:101E9000B440E4430294541E012C2AD88768029C63
:101EA0002740CC68B4403C43846044680127AC437D
:101EB0002500644624093C409C402C434460C5688E
:101EC000029C25408C68B4402C43C460022A12D185
:101ED000DC080725A4000419276A03940F241D4079
:101EE000AD00AC40A7430C69AC402743039C27627C
:101EF00001E0032AE3D10468029DB24025402C0092
:101F000014430460C0246246A40222424FD001253B
:101F1000284A90279469FF052C43946192699C0894
:101F20002A400592059A244AA400A4180F220235DB
:101F30001D40AD00AA40A66896430022B8420CD0CE
:101F40001E4F0132B84208D01D4F0132B84204D0B2
:101F50001C4F0132B84200D00232AA4067463243D9
:101F6000A260194A019C1668019DE4433543FF03B2
:101F700001D435002540674615605668019D3543FC
:101F8000BF0301D435002540674655609668019D22
:101F90003543FF0201D43500254067469560D5687A
:101FA000019E2E43BF0201D425402E00D66001338E
:101FB00059E7C046001002400000014000040048FC
:101FC00000080048000C0048000401400069084077
:101FD000431E9841C0B27047002A01D0816170470A
:101FE0008162FCE7426913000B401B0491431943D3
:101FF00081617047044B10B55A69104202D0586194
:10200000FFF70CF810BDC0460004014070B5040095
:102010000120002C17D02368124A07251A60124AA3
:102020001A6062685A60A2689A60FFF78BF906002E
:102030002368DA68100028402A4205D11969E2684D
:1020400091420CD01A6170BDFFF77CF9801B2728E4
:10205000EED92368DB682B42EAD00320F3E7034A7A
:102060001A60F0E7CCCC000055550000AAAA000089
:102070000368024A00201A607047C046AAAA0000FE
:10208000F0B5040085B0002845D00368DB072FD4E5
:1020900023689B0700D581E023681B0700D5BCE0BF
:1020A00023685B0700D5DFE02368DB061AD5626989
:1020B0000423B54D012A00D04AE1696B02270B4386
:1020C0006B636B6B1A436A63FFF73CF906006B6B3B
:1020D0003B4200D135E1F8216A6BA3698A43DB00FA
:1020E00013436B63236A002B00D059E100202AE0E0
:1020F0000C21A54D6A680A40042A06D06B680B4083
:10210000082B0AD16B68DB0307D52B689B03BFD56F
:102110006368002BBCD1012015E06368012B14D14A
:1021200080232A685B0213432B60FFF70BF980279B
:102130000600BF022B683B42AAD1FFF703F9801BC0
:102140006428F7D9032005B0F0BD002B16D12B6809
:102150008E4A802713402B602B688D4ABF021340A4
:102160002B60FFF7EFF806002B683B4200D18FE7AA
:10217000FFF7E8F8801B6428F6D9E3E7052B05D1C3
:1021800080232A68DB0213432B60C9E72B687F4A50
:1021900013402B602B687E4A1340C5E70C227A4D12
:1021A0006B68134206D06B681340082B10D16B6824
:1021B000DB030DD42B689B0702D5E368012BAAD162
:1021C000F8212A6823698A43DB0013432B6063E705
:1021D000E2680123002A0FD02A68022713432B60EC
:1021E000FFF7B0F806002B683B42E9D1FFF7AAF8E9
:1021F000801B0228F7D9A5E72A6802279A432A609C
:10220000FFF7A0F806002B683B4200D144E7FFF738
:1022100099F8801B0228F6D994E7E26901235A4D08
:10222000002A10D06A6A022713436B62FFF78AF80C
:1022300006006B6A3B4200D032E7FFF783F8801B51
:102240000228F6D97EE76A6A02279A436A62FFF794
:1022500079F806006B6A3B4200D121E7FFF772F87C
:10226000801B0228F6D96DE780220021464D5205D9
:10227000EB690091134208D1EB691343EB61EB6901
:1022800013400393039B012300938027414E7F005B
:1022900033683B4206D0A368012B13D12A6A13434B
:1022A0002B6230E033683B433360FFF74BF801901B
:1022B00033683B42EFD1FFF745F8019BC01A642811
:1022C000F6D93FE70122002B14D12B6A0227934352
:1022D0002B622B6A033293432B62FFF733F806001D
:1022E0002B6A3B4216D0FFF72DF82B4B801B9842F0
:1022F000F6D927E7052B16D1296A013B0B432B6240
:102300002B6A1A432A62FFF71DF8022706002B6A80
:102310003B420FD0009B012B00D0C5E6EB691F4A62
:102320001340EB61C0E62B6A934304222B622B6AB5
:102330009343B5E7FFF706F8174B801B9842E6D9A1
:1023400000E7FEF7FFFF801B022800D8BFE6F9E692
:10235000053203D16A6B9A436A63BCE66A6B022753
:10236000134301226B636B6B93436B63FEF7EAFFCE
:1023700006006B6B3B4200D1B4E6FEF7E3FF801B27
:102380000228F6D9DEE6C04600100240FFFFFEFF3D
:10239000FFFFFBFF0070004088130000FFFFFFEF0E
:1023A0000C21344D6A680A40082A47D0324A022B71
:1023B00032D12B68802713402B60FEF7C3FF060045
:1023C000BF042B683B4221D10F22EB6A8026934346
:1023D000E26AB6041343EB62616AA36A6A680B435C
:1023E00026490A4013436B6080232A685B04134329
:1023F0002B60FEF7A7FF04002B68334200D075E680
:10240000FEF7A0FF001B0228F6D99BE6FEF79AFF15
:10241000801B0228D5D995E62B68802613402B60B7
:10242000FEF790FF0400B6042B68334200D15DE64E
:10243000FEF788FF001B0228F6D983E61800012B5F
:1024400000D180E680216B68606A4902EA6A19401F
:10245000814200D05FE60F210A40E16A8A4200D043
:1024600059E6F02292031340A26A934200D13DE65E
:1024700051E6C04600100240FFFFFFFEFFFFC2FF13
:1024800070B588B010221249684604AD01F0CEF94B
:10249000102228000F4901F0C9F90C220E4E736872
:1024A0001A40082A11D10F206A46990C0140545C49
:1024B000F26A0240A95CDB0305D50848FDF740FE3F
:1024C000604308B070BD0648FAE70448F9E7C04623
:1024D000923A0008A33A00080010024000127A0065
:1024E00000093D00F7B504000E00002801D10120CD
:1024F000FEBD0122374D2B6813408B421CD321684F
:102500008B0722D4CB072FD401232A681A40B2426A
:1025100051D82368304D5B0754D4FFF7B1FF6B6887
:102520002E4A1B061B0FD35CD8402D4B186003208E
:10253000FEF7D4FE0020DBE72B6893430B432B60B0
:102540002B6813408B42D2D1D9E7234A4B0704D5DD
:10255000E0235068DB0003435360F020536883435B
:10256000A06803435360CDE71B4F62683B68012AB4
:1025700019D19B03BBD503217B688B4313437B603D
:10258000FEF7E0FE01900C237A681A4063689B0016
:102590009A42B9D0FEF7D6FE019BC01A114B984261
:1025A000F1D90320A4E7022A02D19B01E3D49EE7DC
:1025B0009B07E0D49BE72A689A432A602A681A425C
:1025C000A7D094E76B68084A1340E26813436B6036
:1025D000A3E7C0460020024000100240683800080F
:1025E0000000002088130000FFF8FFFF044B054A9D
:1025F0005B685B055B0FD35C034A1068D84070478B
:10260000001002407838000800000020F0B5036890
:10261000050085B0DB032AD580220021384C520505
:10262000E3690091134208D1E3691343E361E3696D
:1026300013400393039B012300938027314E7F00B7
:1026400033683B4228D0226AC02311009B002E4EE3
:1026500019401A4232D1236A1E406B681E43009B08
:102660002662012B03D1E369284A1340E3612A68FB
:10267000D30706D5032022490B6B8343A868034385
:102680000B630020930617D510211D4A136B8B4353
:10269000E9680B4313630FE033683B433360FEF795
:1026A00051FE019033683B42CDD1FEF74BFE019BBA
:1026B000C01A6428F6D9032005B0F0BD6A6813403B
:1026C0008B42C8D08023226A206A11005B02034338
:1026D0002362236A0E483140034023622162D307FC
:1026E000B9D5FEF72FFE07000222236A1342B2D1AA
:1026F000FEF728FE074BC01B9842F5D9DBE7C04622
:102700000010024000700040FFFCFFFFFFFFFFEFE2
:10271000FFFFFEFF881300000122036A70B5934398
:102720000362036A44688569723295430A681543F7
:10273000022293438A681343114A904205D0114EF6
:10274000B04202D0104EB04213D10826B343CE6837
:1027500033430426B343904205D00A4A904202D044
:10276000094A904205D1094A8E6922404C69344396
:1027700014434A68446085614263036270BDC04689
:10278000002C01400044014000480140FFFCFFFFD5
:1027900070B57325036A164A13400362036A4268E0
:1027A000C469AC430D682C43124D2B408D682D023B
:1027B0002B43114DA8420ED1104D1D40CB681B027A
:1027C0002B430F4D2B400F4D4E6915408A69324304
:1027D00012012A4305E00C4DA842F4D00B4DA8424B
:1027E000F1D042604A68C461C263036270BDC046F2
:1027F000FFFEFFFFFFFDFFFF002C0140FFF7FFFF83
:10280000FFFBFFFFFFCFFFFF0044014000480140F6
:10281000036A124A30B513400362026A104C4368DF
:10282000C56925400C68240225430E4C22408C6863
:10283000240322430C4CA04205D00C4CA04202D0F1
:102840000B4CA04204D10B4C23404C69A401234300
:1028500043604B68C5610364026230BDFFEFFFFF58
:10286000FF8CFFFFFFDFFFFF002C01400044014011
:1028700000480140FFBFFFFF0200030001203D327E
:102880001178814215D1022111701B68DA68024368
:10289000DA600B4A934202D00A4A93420AD10721D6
:1028A0009A6800200A40062A03D0012219680A43C8
:1028B0001A6070471A68104318600020F9E7C04694
:1028C000002C01400004004070477047704770477B
:1028D000704770470222036810B51969040011425D
:1028E0000ED0D96811420BD0053A1A610432027732
:1028F0009B699B0700D179E0FFF7E9FF002323776D
:10290000042223681969114210D0D96811420DD0F0
:10291000093A1A61073222779A69C0239B00200086
:102920001A4269D0FFF7D3FF0023237708222368D8
:10293000196911420ED0D96811420BD0113A1A61AF
:102940000D322277DB6920009B075BD0FFF7BFFFCA
:1029500000232377102223681969114210D0D96807
:1029600011420DD0213A1A6119322277DA69C02357
:102970009B0020001A424BD0FFF7A9FF00232377CA
:10298000012223681969114207D0D968114204D085
:10299000033A20001A61FFF798FF80222368196923
:1029A000114208D0D968114205D0023AFF3A2000FE
:1029B0001A6100F0DCF9402223681969114207D03E
:1029C000D968114204D0813A20001A61FFF781FFD3
:1029D000202223681969114207D0D968114204D016
:1029E000413A20001A6100F0C1F910BDFFF76EFFF7
:1029F0002000FFF76DFF81E7FFF768FF2000FFF77A
:102A000067FF91E7FFF762FF2000FFF761FF9FE795
:102A1000FFF75CFF2000FFF75BFFAFE7194A10B537
:102A20000368904202D0184CA04208D17024A343FE
:102A30004C68234390420BD0134CA04208D0134C57
:102A4000A04205D0124CA04202D0124CA04203D1A9
:102A5000114C2340CC6823438024A3434C69234377
:102A600003608B68C3620B688362904205D0084B99
:102A7000984202D0074B984201D10B6903630123AE
:102A8000436110BD002C01400004004000200040C4
:102A90000044014000480140FFFCFFFF70B5040006
:102AA0000120002C21D025003D352B78DAB2002BF7
:102AB00005D123003C3320001A70FDF76BFF022381
:102AC0002B702068211DFFF7A9FF220001230020A1
:102AD000463213704534083A137053709370D370B4
:102AE00013715371937123702B7070BD70B5040016
:102AF0000120002C21D025003D352B78DAB2002BA7
:102B000005D123003C3320001A70FFF7DDFE0223BD
:102B10002B702068211DFFF781FF22000123002078
:102B2000463213704534083A137053709370D37063
:102B300013715371937123702B7070BD1022036A4F
:102B400070B593430362026A154C4368856925405A
:102B50000C68240225432024A2438C6824012243CC
:102B6000104CA0420FD18024A2431400CA68120165
:102B700022434024A2430C4E4C691E408B692343E0
:102B80009B00334305E0094CA042F4D0084CA0421E
:102B9000F1D043604B6885618363026270BDC046BB
:102BA000FF8CFFFF002C0140FFF3FFFF00440140BA
:102BB00000480140F8B507003C373B7804000E00A0
:102BC00015000220012B0AD001383870082A3DD0A8
:102BD00006D8002A17D0042A27D000233B70F8BD5E
:102BE0000C2AFAD12068FFF713FE80222368120115
:102BF000D9690A43DA61DA691C490A40DA61326943
:102C0000D96912022FE02068FFF786FD08222368A9
:102C100099690A4304219A619A698A439A619A6977
:102C200031690A439A610020D7E72068FFF786FFE1
:102C300080222368120199690A439A619A690B49B3
:102C40000A409A61326999691202EAE72068FFF73F
:102C50009FFD04212368DA691543DD61DA698A433F
:102C6000DA61DA6931690A43DA61DCE7FFFBFFFF09
:102C70001F2310B5012419408C408A40036AA343E6
:102C80000362036A1A43026210BD000010B504001B
:102C9000002906D1020001203E321378834238D049
:102CA00010BD030004292ED13F331B780120013BC6
:102CB0005A1E9341DBB2002BF2D1022322000429D9
:102CC0002DD13F3213702268D3680B43D360206844
:102CD0000122FFF7CDFF23681E498B422CD01E4AEC
:102CE000934229D01D4A934226D01D4A93422BD1AC
:102CF00007219A6800200A40062AD1D001221968CB
:102D00000A431A60CCE7082901D14033CDE74133AB
:102D1000CBE7022313702268D0680343D6E7082963
:102D200001D14032CEE74132012013700C29B7D1D6
:102D300022681023D068F0E78022586C1202024308
:102D40005A648B42D1D1D3E70122196800200A438B
:102D50001A60A5E7002C01400044014000480140F2
:102D60000004004010B5FFF791FF10BD7047704799
:102D700030B5EFF31084012282F310880168124D00
:102D80000B682B400B6084F31088EFF3108482F300
:102D9000108801688B6893438B6084F31088036EFE
:102DA00093420AD1EFF3108183F310881024026854
:102DB0001368A343136081F310882023C3670023A3
:102DC0000366436630BDC046DFFEFFFFF7B5130064
:102DD000826F04000220202A3AD10138002937D01E
:102DE000002B35D08022A0685201904206D1226982
:102DF000002A03D101321000114229D12500743577
:102E00002A780220012A23D001222A70220050327F
:102E1000E1640026138053802122E06E271DFE67A7
:102E2000A267B04215D0226846630192124A8262BC
:102E3000124AC262124A0263019A2832FEF72CFE3D
:102E4000B04206D010230120FB67DB182E70A36769
:102E5000FEBD4022002023681A622870EFF3108123
:102E6000012383F3108822687F339468234393609F
:102E700081F31088ECE7C046392F0008852F000841
:102E8000952F00088021026870B5836FC56F926826
:102E900004000A422BD0212B29D1EFF31080203BD4
:102EA00083F31088226893688B43936080F31088C3
:102EB000E06E00280DD0FEF72DFE002809D0E06E50
:102EC000FEF7B6FE202804D110230434E3671D3832
:102ED00070BDEFF31081012383F31088C0202268B6
:102EE00013688343136081F310882023A367402174
:102EF000236800209B680B42EAD0222DE8D1EFF333
:102F00001080012383F31088226893688B439360B9
:102F100080F31088206F002808D0FEF7FBFD002802
:102F200004D0206FFEF784FE2028CDD02000FFF7CC
:102F30001FFF0020CCE7704703009B6970B5406A13
:102F4000202B1BD00300002252331A80EFF3108491
:102F5000013282F31088802501688B68AB438B6057
:102F600084F31088EFF3108182F310884023026805
:102F700010680343136081F3108870BDFFF7DBFF17
:102F8000FBE7704710B5406AFFF7FBFF10BD7047C5
:102F90007047704770B5446A2268A36FE16F92680A
:102FA000120613D5212B11D12300002252331A808F
:102FB000EFF31080012383F31088C0252268136883
:102FC000AB43136080F310882023A36723689B68BA
:102FD0005B0608D5222906D1230000225A3320009F
:102FE0001A80FFF7C5FE1023221DD16F20000B436E
:102FF000D367FFF7CEFF70BD406A0023020010B513
:103000005A321380083A1380FFF7C3FF10BD704790
:103010000168F8B5CB699F4D040008688A682B42A7
:103020000BD12022134200D17EE0104200D17BE080
:10303000636E2000002B6DD16DE00126964D32406D
:103040000540154300D16FE0251D334205D0C7056B
:1030500003D50E62EF6F3E43EE670226334206D081
:10306000002A04D00E62EF6FB6193E43EE670426C5
:10307000334206D0002A04D00E62EF6F023E3E4378
:10308000EE670826334207D0202707403A4303D093
:103090000E62EA6F1643EE6780221201134206D0D9
:1030A000460104D50A622022E96F0A43EA67EA6F03
:1030B000002A30D02022134206D0104204D0636E82
:1030C000002B01D0200098472268EB6F40279668BC
:1030D00028223E40134020001E4321D0FFF748FE27
:1030E00023689B683B4217D0EFF31081012383F3E1
:1030F000108822689368BB43936081F31088206F27
:10310000002809D0654B4363FEF722FD002802D05A
:10311000206F436B9847F8BD2000FFF73AFFFAE7AE
:10312000FFF737FFEE67F6E7226E012A00D090E046
:1031300010252B4200D18CE0284200D189E00D629D
:103140008B684021180008400B424CD0206F036868
:103150005B689BB2002BDED02600583637889F4232
:10316000D9D927005A373B808369202B31D0EFF320
:10317000108782F310882068494D03682B40036054
:1031800087F31088EFF3108782F310882068836834
:103190009343836087F31088EFF3108782F31088DE
:1031A000206883688B43836087F310882023E3675C
:1031B00000232366EFF3108182F310882268123512
:1031C0001368FF35AB43136081F31088206FFEF75F
:1031D000A1FC23005A331B883188C91A89B2200008
:1031E000FFF715FF97E726005A36338831889BB2E0
:1031F000002900D18FE7210058310988C91A89B206
:10320000002900D187E7EFF3108782F31088266842
:10321000244D33682B40336087F31088EFF3108719
:1032200082F310882668B3689343B36087F31088ED
:1032300020236066E3672066EFF3108082F3108836
:10324000226832351368FF35AB43136080F3108872
:10325000C5E78022134203D0104201D0A36EE8E6F6
:103260004022134200D156E7104200D153E7EFF35A
:103270001080012383F3108821680B6893430B604F
:1032800080F310882023A36700232000A366FFF7A4
:1032900052FE40E70F08000020010004F92F00084B
:1032A000FFFEFFFFDFFEFFFF406A10B5036E012B3C
:1032B00006D10300583319884908FFF7A8FE10BD4E
:1032C000FFF766FEFBE7000003009B6970B5406AEC
:1032D000202B34D0030000225A331A80EFF31084DD
:1032E000012383F3108801681B4D0A682A400A6095
:1032F00084F31088EFF3108483F3108801688A68E0
:103300009A438A6084F31088EFF3108183F3108866
:10331000402402689368A343936081F310882023BC
:10332000C367036E012B0AD1EFF3108183F310887A
:103330000268303C1368A343136081F31088036E66
:10334000012B05D1030058331988FFF760FE70BDCB
:10335000FFF71DFEFBE7C046FFFEFFFF70B5040050
:103360002569A26801682A436569C3692A43086818
:10337000394D1A43284002430A604A683748256A93
:103380000240E06802434A60A26988682A43344DDB
:10339000284002438A600321324A126B0A4080218E
:1033A000013A0902022A4CD82F48805C8B4224D172
:1033B000082817D8FCF7BAFE471608160516161681
:1033C0000900FFF75DF840E0284B5800636861682A
:1033D0005B08C018FCF7B4FE254982B2103A03041A
:1033E0008A4201D9012033E00F221B03904380B2AF
:1033F00022685B0F1843D06029E00828F2D8FCF758
:103400008BFE16F11EF11BF1F1F105008020000288
:10341000636861685B081818FCF792FE80B20200CE
:10342000134B103A9A42DDD82368D8600FE0FFF7BB
:10343000DDF800280BD0EBE7FFF722F8F9E70B489F
:10344000E6E78B42F3D1FFF7D1F8031EBDD1002090
:1034500000236366A36670BDF369FFFFFFCFFFFF24
:10346000FFF4FFFF00100240B43A000800127A0097
:10347000EFFF0000436A30B5DA0706D50168284C33
:103480004A682240846A22434A609A0706D5016846
:10349000244C4A682240C46A22434A605A0706D52F
:1034A0000168214C4A682240046B22434A601A0793
:1034B00006D501681D4C4A682240446B22434A608D
:1034C000DA0606D501681A4C8A682240846B2243CA
:1034D0008A609A0606D50168164C8A682240C46B39
:1034E00022438A605A0610D50168134D4A68046C5D
:1034F0002A4022434A6080225203944205D14A68FE
:103500000E4C2240446C22434A601B0606D50268DA
:103510000B4953680B40816C0B43536030BDC04670
:10352000FFFFFDFFFFFFFEFFFFFFFBFFFF7FFFFF32
:10353000FFEFFFFFFFDFFFFFFFFFEFFFFFFF9FFF3B
:10354000FFFFF7FFF7B5802704000D001600019379
:103550003F012268D3692B405B1B59424B41B34268
:1035600001D0002028E0089B0133F3D0FDF7EAFEEC
:10357000019BC01A089B984201D8002B1DD1EFF384
:103580001080012282F3108821681E4D0B682B40A9
:103590000B6080F31088EFF3108082F310882168AD
:1035A0008B6893438B6080F310882023A367E367C5
:1035B0000023032074342370FEBD042123681A689D
:1035C0000A42C6D0DA693A42C3D01F62EFF31080D4
:1035D000012282F3108821680A4D0B682B400B6092
:1035E00080F31088EFF3108082F3108821688B68D5
:1035F00093438B6080F310882023221DA367E36729
:10360000D367D5E75FFEFFFF73B500260400031DF7
:10361000DE67FDF797FE236805001B681B0716D4BD
:1036200023681B685B070AD580210F4B002200939B
:1036300020002B00C903FFF785FF002812D12023AB
:103640000020A367E3672066743420700BE08021BC
:10365000054B32000093890303002000FFF772FF3F
:103660000028DDD0032076BDFFFFFF0110B5041E4A
:1036700001D1012010BD836F002B04D102007432F0
:103680001370FDF71FFA242301212268A367136832
:1036900020008B431360FFF761FE0128E9D0636AC5
:1036A000002B02D02000FFF7E5FE236807495A6887
:1036B00020000A4008215A609A688A439A600122D1
:1036C00019680A431A60FFF79FFFD3E7FFF7FFFF70
:1036D000F8B513000200040058324165002513803C
:1036E00022222600071DFD67C267006F7436A842BC
:1036F00016D01E4A456382621D4AC2621D4A026399
:103700002268243294460A006146FEF7C5F9A842B1
:1037100006D010230120FB67DB183570E367F8BD86
:1037200000203070EFF31085012383F3108880228E
:10373000216852000E6832430A6085F31088EFF367
:10374000108583F3108821688A681A438A6085F39C
:103750001088EFF3108183F3108822683F33946858
:103760002343936081F31088D9E7C046C93200082B
:10377000A9320008952F000870B5C46F0223202CD1
:103780002DD1013B00292AD0002A28D0802384682B
:103790005B019C4206D10369002B03D10124230065
:1037A00021421CD10400743425780223012D16D047
:1037B000013B2370002404660468646824020BD56E
:1037C000EFF3108583F3108880230468DB042668F8
:1037D0003343236085F31088FFF77AFF0300180056
:1037E00070BD000070B500260C4D0D4C641BA4107C
:1037F000A64209D1002600F02BF80A4D0A4C641BA2
:10380000A410A64205D170BDB300EB58984701360D
:10381000EEE7B300EB5898470136F2E7B83A0008F4
:10382000B83A0008B83A0008BC3A0008002310B5BE
:103830009A4200D110BDCC5CC4540133F8E70300B8
:103840008218934200D1704719700133F9E70000E4
:10385000F8B5C046F8BC08BC9E467047F8B5C046EF
:08386000F8BC08BC9E4670474D
:103868000000000000000000010203040607080928
:1038780000000000010203044443452D3233303276
:103888002D56342E335F48414C0000C1814001C0A1
:10389800804101C0804100C1814001C0804100C118
:1038A800814000C1814001C0804101C0804100C108
:1038B800814000C1814001C0804100C1814001C0F8
:1038C800804101C0804100C1814001C0804100C1E8
:1038D800814000C1814001C0804100C1814001C0D8
:1038E800804101C0804100C1814000C1814001C0C8
:1038F800804101C0804100C1814001C0804100C1B8
:10390800814000C1814001C0804101C0804100C1A7
:10391800814000C1814001C0804100C1814001C097
:10392800804101C0804100C1814000C1814001C087
:10393800804101C0804100C1814001C0804100C177
:10394800814000C1814001C0804100C1814001C067
:10395800804101C0804100C1814001C0804100C157
:10396800814000C1814001C0804101C0804100C147
:10397800814000C1814001C0804100C1814001C037
:10398800804101C0804100C1814000C0C101C30322
:1039980002C2C60607C705C5C404CC0C0DCD0FCF9F
:1039A800CE0E0ACACB0BC90908C8D81819D91BDB0F
:1039B800DA1A1EDEDF1FDD1D1CDC14D4D515D7175F
:1039C80016D6D21213D311D1D010F03031F133F30F
:1039D800F23236F6F737F53534F43CFCFD3DFF3F5F
:1039E8003EFEFA3A3BFB39F9F83828E8E929EB2B8F
:1039F8002AEAEE2E2FEF2DEDEC2CE42425E527E71F
:103A0800E62622E2E323E12120E0A06061A163A38E
:103A1800A26266A6A767A56564A46CACAD6DAF6F1E
:103A28006EAEAA6A6BAB69A9A86878B8B979BB7B8E
:103A38007ABABE7E7FBF7DBDBC7CB47475B577B7DE
:103A4800B67672B2B373B17170B05090915193530E
:103A5800529296565797559594549C5C5D9D5F9FDE
:103A68009E5E5A9A9B5B99595898884849894B8B0E
:103A78008A4A4E8E8F4F8D4D4C8C4484854587479E
:103A8800468682424383418180400203040506073B
:103A980008090A0B0C0D0E0F101000010203040593
:103AA800060708090A0B0C0D0E0F10000408020087
:043AB800E900000819
:043ABC00C10000083D
:103AC00000127A000100460001010000040000001D
:040000050800128954
:00000001FF
